:100000000C9425050C946C050C946C050C946C05F3
:100010000C946C050C946C050C946C050C946C059C
:100020000C946C050C946C050C94B50C0C946C053C
:100030000C945F1B0C946C050C946C050C946C0573
:100040000C946C050C946C050C946C050C946C056C
:100050000C946C050C94FF1B0C946C050C946C05B3
:100060000C946C050C946C050C946C050C946C054C
:100070000C946C050C946C050C946C050C946C053C
:100080000C946C050C946C050C946C050C946C052C
:100090000C946C050C946C050C946C050C946C051C
:1000A0000C946C050C946C050C946C05AB0DCD0D8B
:1000B000BB0ECD0DBB0E120E350EBB0E8A0E9D0E65
:1000C000A211A211CF11CF112A1266125E145E1472
:1000D0007E125E147913791334145E145E144A147C
:1000E0008080352B787939808080210877060780D9
:1000F0008080201A7A1B168080801E802980808054
:100100008080808080808080808022158019098096
:1001100080801F147B1D0480808023172C050A809B
:100120008080260C00360E808080251876100D8089
:100130008080241C80110B80808027127E370F80E6
:1001400080802A804F7D2880808074305152328098
:1001500080802D137C38338080802E2F5075348022
:10016000253032583A20253038620A000A722F634F
:100170002030313233343536370A005B735D004B43
:100180006579626F6172642073746172742E0A0003
:1001900055534220636F6E666967757265642E0AF7
:1001A000005B575D005B535D005B525D005B445D2F
:1001B000005B435D001203480048004B00420020F2
:1001C000006D006F00640000000E0374002E006DCF
:1001D000002E006B002E0000000403090409028DAC
:1001E00000050100A032090400000103010100091B
:1001F00021110100012240000705810308000A09BE
:100200000401000103010200092111010001224D36
:10021000000705820308000A090402000103000028
:10022000000921110100012236000705830308009F
:100230000A09040300020300000009211101000162
:100240002222000705840320000107050403200083
:10025000010904040001030000000921110100014B
:10026000223900070585032000011201100100005A
:100270000008EDFEFECA04010102000105010906A5
:10028000A101050719E029E7150025019508750169
:10029000810205081901290595057501910295014D
:1002A000750391010507190029F71500250195F837
:1002B00075018102C00631FF0974A101097515009D
:1002C00026FF009520750881020976150026FF009B
:1002D000952075089102C005010980A101850216CB
:1002E000010026B7001A01002AB700751095018198
:1002F00000C0050C0901A1018503160100269C021E
:100300001A01002A9C02751095018100C00501099F
:1003100002A1010901A100050919012905150025FE
:10032000019505750181029501750381010501099A
:100330003009311581257F95027508810609381528
:1003400081257F950175088106050C0A3802158103
:10035000257F950175088106C0C005010906A10128
:10036000050719E029E715002501950875018102A7
:100370009501750881010508190129059505750183
:1003800091029501750391010507190029FF1500D8
:1003900026FF00950675088100C00A0025303258F6
:1003A00020006B6579626F6172645F7265706F7255
:1003B000743A20004C45443A20253032580A0064F3
:1003C000656C5F6B65795F6269743A2063616E2763
:1003D000742064656C3A20253032580A00616464E8
:1003E0005F6B65795F6269743A2063616E27742080
:1003F0006164643A20253032580A004F6E65736894
:100400006F743A2074696D656F75740A00290A006B
:100410002575002F002575005D280025640020004B
:10042000256400200025640020002564007C002550
:10043000303258006D6F7573656B6579205B62743F
:100440006E7C782079207620685D287265702F6137
:10045000636C293A205B006D6B5F776865656C5F44
:1004600074696D655F746F5F6D6178203D202564F0
:100470000A006D6B5F776865656C5F6D61785F73AF
:1004800070656564203D2025640A006D6B5F7469AA
:100490006D655F746F5F6D6178203D2025640A0093
:1004A0006D6B5F6D61785F7370656564203D2025BD
:1004B000640A006D6B5F696E74657276616C203DD5
:1004C0002025640A006D6B5F64656C6179203D20B6
:1004D00025640A006D6B5F776865656C5F74696D94
:1004E000655F746F5F6D6178203D2025640A006D43
:1004F0006B5F776865656C5F6D61785F737065656C
:1005000064203D2025640A006D6B5F74696D655F32
:10051000746F5F6D6178203D2025640A006D6B5F0C
:100520006D61785F7370656564203D2025640A0005
:100530006D6B5F696E74657276616C203D20256419
:100540000A006D6B5F64656C6179203D2025640A4B
:10055000000A00257500363A20776865656C5F747F
:10056000696D655F746F5F6D61783A20000A0025E0
:100570007500353A20776865656C5F6D61785F73EB
:10058000706565643A20000A00257500343A2074CD
:10059000696D655F746F5F6D61783A20000A0025B0
:1005A0007500333A206D61785F73706565643A2039
:1005B000000A00257500323A20696E746572766112
:1005C0006C286D73293A20000A00257500313A2005
:1005D00064656C6179282A31306D73293A20000AEC
:1005E000092D2056616C756573202D0A004D3E0063
:1005F0004D25643E20003F0073657420646566618C
:10060000756C740A00433E2000776865726520644B
:10061000656C74613A20637572736F723D25642C4A
:1006200020776865656C3D25640A536565206874AC
:1006300074703A2F2F656E2E77696B6970656469E7
:10064000612E6F72672F77696B692F4D6F757365B8
:100650005F6B6579730A000A092D204D6F7573650C
:100660006B6579202D0A4553432F713A09717569DD
:10067000740A313A0964656C6179282A31306D73E6
:10068000290A323A09696E74657276616C286D7355
:10069000290A333A096D61785F73706565640A34BD
:1006A0003A0974696D655F746F5F6D61780A353AF8
:1006B00009776865656C5F6D61785F737065656407
:1006C0000A363A09776865656C5F74696D655F74B1
:1006D0006F5F6D61780A0A703A097072696E7420F2
:1006E00076616C7565730A643A0973657420646594
:1006F0006661756C74730A75703A092B310A646F00
:10070000776E3A092D310A706775703A092B3130CE
:100710000A7067646F776E3A092D31300A0A737078
:10072000656564203D2064656C7461202A206D61DC
:10073000785F7370656564202A2028726570656132
:1007400074202F2074696D655F746F5F6D61782907
:100750000A003F004D3E2000433E20004C25640A25
:10076000000A092D20436F6E736F6C65202D0A45BA
:1007700053432F713A09717569740A6D3A096D6FA7
:100780007573656B65790A000A092D204D616769EB
:1007900063202D0A643A0964656275670A783A092C
:1007A0006465627567206D61747269780A6B3A09D5
:1007B0006465627567206B6579626F6172640A6D4A
:1007C0003A096465627567206D6F7573650A763ADC
:1007D0000976657273696F6E0A733A09737461748E
:1007E00075730A633A09636F6E736F6C65206D6F82
:1007F00064650A302D343A096C61796572302D34A4
:10080000284631302D4634290A506175733A096201
:100810006F6F746C6F616465720A6E3A094E4B5269
:100820004F0A003F004E4B524F3A206F66660A0057
:100830004E4B524F3A206F6E0A0074696D65725FBD
:1008400072656164333228293A202530346C580AA5
:10085000006B6579626F6172645F6E6B726F3A20D4
:1008600025580A006B6579626F6172645F69646C18
:10087000653A2025580A006B6579626F6172645F82
:1008800070726F746F636F6C3A2025580A00686F3E
:1008900073745F6B6579626F6172645F6C656473BA
:1008A00028293A2025580A000A092D20537461741A
:1008B0007573202D0A004743433A20342E392E32D7
:1008C000204156522D4C4942433A20312E382E3089
:1008D00073766E204156525F415243483A2061760A
:1008E00072350A004F5054494F4E533A204C5546EA
:1008F00041204D4F5553454B455920455854524181
:100900004B455920434F4E534F4C4520434F4D4D7F
:10091000414E44204E4B524F204B45594D41505F64
:1009200053454354494F4E20343039360A0042551E
:10093000494C443A203038646361313220283039E0
:100940003A35303A34302053657020203720323029
:100950003136290A005649443A2030784645454404
:1009600028742E6D2E6B2E29205049443A20307861
:10097000434146452848484B42206D6F6429205624
:1009800045523A203078303130340A0044455343E0
:100990003A20742E6D2E6B2E206B6579626F61721A
:1009A00064206669726D7761726520666F72204897
:1009B000484B42206D6F640A000A092D205665726B
:1009C00073696F6E202D0A000A6D6F7573653A208A
:1009D0006F66660A000A6D6F7573653A206F6E0A5E
:1009E000000A6B6579626F6172643A206F66660A0D
:1009F000000A6B6579626F6172643A206F6E0A005B
:100A00000A6D61747269783A206F66660A000A6D31
:100A100061747269783A206F6E0A000A64656275C3
:100A2000673A206F6E0A000A64656275673A206F44
:100A300066660A000A0A626F6F746C6F61646572A1
:100A40002E2E2E2000433E20000011241FBECFEF8B
:100A5000DAE0DEBFCDBF04B603FE27C080912102DD
:100A600090912202A0912302B09124028730904BF2
:100A7000A740B04BD1F410922102109222021092A2
:100A800023021092240214BE84B7877F84BF0FB65E
:100A9000F894A8958091600088618093600010921E
:100AA00060000FBEE0E0F8E3099511E0A0E0B1E0DE
:100AB000E8E1F9E402C005900D92A833B107D9F737
:100AC00022E0A8E3B1E001C01D92A132B207E1F734
:100AD0000E94DD090C948A240C940000FF93EF938C
:100AE000E0913801F0913901309709F00995EF91C3
:100AF000FF910895FC018591803011F0EFDFFBCF6D
:100B00000895FF27E0E230E247FF0CC0419597FFD0
:100B100009C0EDE26095709580959095611D711DFD
:100B2000811D911D27FF02C0219530E350E2AA27C5
:100B3000660F771F881F991FAA1FA41710F0A41B08
:100B400063955A95A9F7AA3008F0A95FA05DAF9305
:100B5000F395611571058105910541F7ED3211F4A9
:100B6000EF93F395F21718F43F93F395FBCF8F9122
:100B7000B5DFFA95E1F70895E991F9918591803013
:100B800021F0853219F0AADFF9CF089520E0E8942A
:100B900055915532C1F3503311F4689455915A333D
:100BA00048F4505390F3220F022E220F220F200DF3
:100BB000250FF4CF0EF4219589919991533619F3AD
:100BC000533729F1533559F1BC0188279927E89407
:100BD0005C3621F48991999168945591543639F491
:100BE00046EF7EF077FF0DC08FEF9FEF0AC05537BD
:100BF0004AE039F0583540E121F0523642E009F040
:100C00000895FF93EF937DDFEF91FF91B7CFFF93AF
:100C1000EF93FC0181918030B9F360DFFBCFFF934C
:100C2000EF9368DFF1CFDF93CF93CDB7DEB7259693
:100C3000A3DFCF91DF9108958FEF84B980E485B968
:100C400057985F9A87B1806C87B988B1806C88B9F2
:100C50002E9A2F98EAE4F1E080E18E0F11928E1324
:100C6000FDCFEAE3F1E080E18E0F11928E13FDCF0C
:100C70008AE491E090935D0180935C018AE391E0C6
:100C800090935B0180935A010895EF92FF920F9326
:100C90001F93CF93DF9380915A0190915B01209134
:100CA0005C0130915D0130935B0120935A01909378
:100CB0005D0180935C01C0E0D0E001E010E080E0E5
:100CC00090E0FC2FF770EC2FE87025B1207C2F2BE3
:100CD000AC0133E0440F551F3A95E1F7242B25B9B9
:100CE00028B12F73EE2311F0206401C0206828B9C9
:100CF0002AE12A95F1F700C0A0915A01B0915B0159
:100D0000AC0FBD1F2C9130E0082E02C03595279501
:100D10000A94E2F720FD2F9AA5E3AA95F1F70000C7
:100D2000F6B42E98BAE1BA95F1F700C040915C0193
:100D300050915D01BA016C0F7D1F4F9B0BC0980154
:100D4000082E01C0220F0A94EAF72095DB013C919E
:100D5000232309C0DB01EC909801082E01C0220F6B
:100D60000A94EAF72E292C9326B56F2D70E02F15E3
:100D700018F026B530E004C026B530E021503F4FD2
:100D8000261B370B2630310558F0A0915A01B0913F
:100D90005B01AC0FBD1F2C91DA01AC0FBD1F2C9372
:100DA000BAE1BA95F1F700C02F982E9A20EA2A9559
:100DB000F1F701968830910509F087CFA0915C0189
:100DC000B0915D01AC0FBD1FE0915A01F0915B0144
:100DD000EC0FFD1F9C918081981751F00E949D1B84
:100DE00060935E0170935F01809360019093610155
:100DF0002196C031D10509F062CF8091180285306B
:100E000021F080911802811111C060915E017091F2
:100E10005F0180916001909161010E94D31B61315B
:100E200077428105910510F00E94201B81E0DF913F
:100E3000CF911F910F91FF90EF90089520915C0149
:100E400030915D01F901E80FF11D808108950F9344
:100E50001F93CF93DF938CE691E00E947A05C0E068
:100E6000D0E000E611E0E0915C01F0915D01EC0F53
:100E7000FD1F80810E94F61A1F928F93DF93CF93FC
:100E80001F930F930E94130621960F900F900F90BF
:100E90000F900F900F90C031D10529F7DF91CF91BE
:100EA0001F910F91089508950895569A81FF02C0E9
:100EB0005E9A08955E9808958091850108959FB780
:100EC000F894109264019FBF90911802943009F039
:100ED00057C09091E9009F703091EC00232F217052
:100EE00030FD20E8922B24E02093E9002091EB00D4
:100EF00020FF43C02091EE0027FF3FC020916201F8
:100F0000222321F02091E80025FF37C010926201D2
:100F100026E03091E80035FD15C0309118023430DC
:100F200061F53091EB0035FD28C0215021F481E0BE
:100F30008093620122C0EFE9FFE03197F1F700C032
:100F40000000E7CF8093F1008091E80085FD0AC0A2
:100F50008091E80080FFFCCF8091E8008E7780933D
:100F6000E80006C08FB7F89421E0209364018FBF9A
:100F70009F709093E90080E008959F709093E9003E
:100F80008FEF0895CF93DF9300D01F92CDB7DEB7D8
:100F90009C0180911802843019F593E099833B837A
:100FA0002A839093E9008FEF9091E800815095FD9E
:100FB00006C095ED9A95F1F700008111F5CF80916B
:100FC000E80085FF0DC040E050E063E070E0CE0136
:100FD00001960E94A30A8091E8008E778093E80032
:100FE0000F900F900F90DF91CF910895CF93DF93E3
:100FF00000D01F92CDB7DEB720911802243021F522
:1010000022E029839B838A8383E08093E9008FEF2A
:101010009091E800815095FD06C095ED9A95F1F705
:1010200000008111F5CF8091E80085FF0DC040E000
:1010300050E063E070E0CE0101960E94A30A809127
:10104000E8008E778093E8000F900F900F90DF916B
:10105000CF910895209118022430F1F422E02093DA
:10106000E9002FEF3091E800215035FD06C035ED45
:101070003A95F1F700002111F5CF2091E80025FF06
:101080000BC040E050E065E070E00E94A30A809150
:10109000E8008E778093E8000895CF93DF93209146
:1010A0001802243009F048C0EC0180910A0188231D
:1010B000E1F080910B018823C1F085E08093E90085
:1010C0008FEF9091E800815095FD06C095E19A95CB
:1010D000F1F700008111F5CF8091E80085FF2CC069
:1010E00040E050E060E270E017C081E08093E900EA
:1010F0008FEF9091E800815095FD06C095ED9A958F
:10110000F1F700008111F5CF8091E80085FF14C050
:1011100040E050E068E070E0CE010E94A30A8091B8
:10112000E8008E778093E80080E2FE01A5E6B1E05A
:1011300001900D928A95E1F7DF91CF91089581EBAF
:1011400091E00E947A0580911702811109C00E94E6
:101150003A0C0E94970C8091E20084608093E20038
:1011600008958DEA91E00E947A0510921702089581
:1011700089EA91E00C947A05209163012F5F822F18
:1011800062E30E945024992319F02093630108958B
:101190001092630180916401882371F1809118029B
:1011A000843041F58091E9008F702091EC00922FFE
:1011B000917020FD90E8892B94E09093E900909144
:1011C000EB0090FF14C09091EE0097FF10C090913B
:1011D000E80095FF03C01092F100F9CF9091E8006C
:1011E00090FF05C09091E8009E779093E8008F7083
:1011F0008093E90010926401089542E061EC81E07F
:101200000E94B40B42E061EC82E00E94B40B42E029
:1012100061EC83E00E94B40B42E261EC84E00E9446
:10122000B40B42E261EC85E00C94B40B80911A029D
:10123000833009F455C030F4813071F0823009F404
:101240008EC008958A3009F47AC08B3009F460C0EA
:10125000893009F09CC020C080911902813A09F0C0
:1012600096C08091E800877F8093E80080911D02FE
:1012700090911E02892B21F460E285E691E003C083
:1012800060E080E090E070E00E94F00A8091E80069
:101290008B778093E800089580911902813209F0DC
:1012A00076C080911D0290911E02009719F004975C
:1012B00009F06DC08091E800877F8093E8008091FD
:1012C000E80082FD05C0809118028111F8CF5FC04F
:1012D0008091F100809385018091E8008B7753C065
:1012E00080911902813A09F052C080911D029091BB
:1012F0001E02892B09F04BC08091E800877F809304
:10130000E8008091E80080FFFCCF80910A0136C0A0
:10131000809119028132D9F580911D0290911E02AF
:10132000892BA9F58091E800877F8093E8000E94CF
:10133000E90B80911B0280930A010C947F14809129
:101340001902813221F58091E800877F8093E800BF
:101350000E94E90B80911C02809386010895809180
:101360001902813AA1F48091E800877F8093E80018
:101370008091E80080FFFCCF809186018093F1008E
:101380008091E8008E778093E8000C94E90B089533
:1013900008950895089585EA91E00E947A050C94D5
:1013A000CA090E94201B80911602882329F00E94FE
:1013B000491B81110C948D0A089584B7877F84BFDF
:1013C0000FB6F894A89580916000886180936000C2
:1013D000109260000FBE90E080E80FB6F894809302
:1013E0006100909361000FBE0E94C8090E94800FA7
:1013F0000E943A0C0E94970C8091E20084608093D6
:10140000E2008FE597E00E94F11A7894809118022B
:10141000843019F00E94D30EF9CF80E991E00E9448
:101420007A050E94820F80E091E00E94EE0E8FE725
:1014300091E00E947A050E94C909809118028530C6
:1014400039F48BE791E00E947A050E94D109F5CF2B
:101450000E94860F0E94D30EF0CF0C945D1B81EA90
:1014600091E00E947A050C942D0A292F332723300E
:101470003105C9F064F42130310581F022303105A5
:1014800009F043C08DE890E02DED31E042C02132FB
:101490003105F1F02232310541F137C082E190E0AF
:1014A0002AE632E036C099278130910541F082303A
:1014B000910541F0892B49F5E9EDF1E005C0E9EC32
:1014C000F1E002C0E5EBF1E0849190E09F0121C0E2
:1014D0006530D8F4E62FF0E0EE0FFF1FED5DFE4F14
:1014E0002081318189E090E014C0653070F470E0B3
:1014F000FB01EE0FFF1FE75EFE4F20813181FB01F4
:10150000EC5EFE4F808190E004C080E090E020E03F
:1015100030E0FA0131832083089580E189BD82E1C2
:1015200089BD09B400FEFDCF8091D8008F7D8093E6
:10153000D8008091E00082608093E0008091E0001C
:1015400081FDFCCF0895CF92DF92EF92FF920F932F
:101550001F93CF93DF93EC018B017A010E94080C5B
:10156000811135C0E114F10439F0F70180819181D6
:10157000081B190BC80FD91FC12CD12C011511053F
:1015800029F18091E80085FD18C08091E8008E77F0
:101590008093E8000E94D30EE114F10449F0F701B2
:1015A00080819181C80ED91ED182C08285E00FC092
:1015B0000E94080C882311F30AC089918093F100DE
:1015C00001501109FFEFCF1ADF0AD8CF80E0DF9179
:1015D000CF911F910F91FF90EF90DF90CF900895E2
:1015E00020911F02309120022617370748F061151D
:1015F000710539F42091E8002E772093E80001C0AE
:10160000B90140E061157105A9F12091180222236A
:1016100009F443C0253009F442C02091E80023FDBD
:1016200040C02091E80022FD32C02091E80020FF58
:10163000E9CF4091F3002091F20030E0342BFC011F
:10164000CF016115710559F02830310540F48191C1
:101650008093F100615071092F5F3F4FF1CF41E05E
:101660002830310509F040E02091E8002E772093E2
:10167000E800C8CF4111C9CF0AC080911802882361
:1016800061F0853061F08091E80083FD0AC08091AF
:10169000E80082FFF2CF80E0089582E0089583E0C1
:1016A000089581E0089520911F02309120022617AD
:1016B000370748F06115710539F42091E8002E775D
:1016C0002093E80001C0B901FC0120E0611571051B
:1016D00091F180911802882309F440C0853009F403
:1016E0003FC08091E80083FD3DC08091E80082FD0D
:1016F0002FC08091E80080FFE9CF2091F300809116
:10170000F20090E0922B6115710559F08830910537
:1017100040F424912093F1003196615071090196B3
:10172000F2CF21E0089709F020E08091E8008E7761
:101730008093E800CBCF2111CCCF0AC08091180252
:10174000882361F0853061F08091E80083FD0AC054
:101750008091E80082FFF2CF80E0089582E0089552
:1017600083E0089581E00895982F973058F590937D
:10177000E900981739F07091EC002091ED0050913C
:10178000F00003C0242F762F50E021FF19C03091C4
:10179000EB003E7F3093EB003091ED003D7F3093C6
:1017A000ED003091EB0031603093EB007093EC0072
:1017B0002093ED005093F0002091EE0027FF07C02A
:1017C0009F5FD3CF8F708093E90081E0089580E020
:1017D00008958091190287FF11C08091E80082FD71
:1017E00005C0809118028111F8CF11C08091E800E6
:1017F0008B770BC080911802882349F08091E80014
:1018000080FFF8CF8091E8008E778093E8000895FC
:101810002091E4003091E50095E64091EC00842FA2
:10182000817040FF22C08091E80080FD1CC0809143
:101830001802882391F0853091F08091EB0085FDAE
:1018400010C04091E4005091E5004217530729F37E
:101850009A01915011F784E0089582E0089583E0A1
:10186000089581E0089580E008954091E80042FFE6
:10187000DECF08950E94A80C0E94B00CE0EEF0E0CC
:10188000808181608083E8EDF0E080818F778083C4
:1018900019BCA7EDB0E08C918E7F8C9380818F7EF8
:1018A00080831092170208950F931F93CF93DF93B5
:1018B0000E94A80C0E94B00CC8EDD0E088818F7700
:1018C000888388818068888388818F7D888319BC1C
:1018D0001092180210921402109216021092150221
:1018E00000EE10E0F80180818B7F80838881816029
:1018F000888342E060E080E00E94B40BE1EEF0E01B
:1019000080818E7F8083E2EEF0E080818160808341
:10191000808188608083F80180818E7F80838881C8
:1019200080618883DF91CF911F910F910895E8ED39
:10193000F0E080818F7E8083E7EDF0E08081816040
:10194000808384E082BF81E0809317020C94540C62
:10195000E8EDF0E080818E7F80831092E2000895B0
:101960001092DA001092E10008951F920F920FB6C4
:101970000F9211242F933F934F935F936F937F9315
:101980008F939F93AF93BF93EF93FF938091E10069
:1019900082FF0BC08091E20082FF07C08091E100CE
:1019A0008B7F8093E1000E94BC088091DA0080FF69
:1019B0001FC08091D80080FF1BC08091DA008E7F0D
:1019C0008093DA008091D90080FF0DC080E189BD4D
:1019D00082E189BD09B400FEFDCF81E08093180249
:1019E0000E949F0805C019BC109218020E94B108FD
:1019F0008091E10080FF19C08091E20080FF15C056
:101A00008091E2008E7F8093E2008091E20080610D
:101A10008093E2008091D80080628093D80019BC46
:101A200085E0809318020E94CB098091E10084FF39
:101A300030C08091E20084FF2CC080E189BD82E14A
:101A400089BD09B400FEFDCF8091D8008F7D8093C1
:101A5000D8008091E1008F7E8093E1008091E200C8
:101A60008F7E8093E2008091E20081608093E200AB
:101A700080911402882311F084E007C08091E30074
:101A800087FD02C081E001C083E0809318020E94BC
:101A90002F0A8091E10083FF24C08091E20083FF40
:101AA00020C08091E100877F8093E10082E08093F5
:101AB0001802109214028091E1008E7F8093E10061
:101AC0008091E2008E7F8093E2008091E20080614D
:101AD0008093E20042E060E080E00E94B40B0E944C
:101AE000B808FF91EF91BF91AF919F918F917F9136
:101AF0006F915F914F913F912F910F900FBE0F907B
:101B00001F9018951F93CF93DF93CDB7DEB7AA9799
:101B10000FB6F894DEBF0FBECDBFE9E1F2E088E07A
:101B20008E0F9091F10091938E13FBCF0E941609B6
:101B30008091E80083FF1FC18091190290911A02E1
:101B4000492F50E04A30510508F015C1FA01EA5A10
:101B5000FF4F0C947024803881F0823809F00BC15B
:101B600080911D028F708093E9008091EB0085FBCE
:101B7000882780F91092E90006C0809115029091A3
:101B80001602911182609091E800977F9093E8008F
:101B90008093F1001092F100C8C0282F2D7F09F02A
:101BA000EAC0882319F0823061F0E5C080911B0201
:101BB000813009F0E0C0933009F080E08093160294
:101BC0002BC080911B02811127C080911D028F7054
:101BD00009F4D1C08093E9002091EB0020FF1CC0E4
:101BE000933021F48091EB00806214C09091EB005F
:101BF00090619093EB0021E030E0A90102C0440F16
:101C0000551F8A95E2F74093EA001092EA0080910E
:101C1000EB0088608093EB001092E9008091E8006F
:101C2000877F86C08111A7C010911B021F7780910A
:101C3000E3008078812B8093E3008091E800877F28
:101C40008093E8000E94E90B8091E80080FFFCCFC0
:101C50008091E30080688093E300111102C082E06C
:101C600001C083E08093180286C08058823008F05B
:101C700082C080911B0290911C028C3D53E095071D
:101C800079F583E08A838AE289834FB7F894DE018D
:101C9000139620E03EE051E2E32FF0E0509357002E
:101CA000E49120FF03C0E295EF703F5FEF708E2F4D
:101CB00090E0EA3010F0C79601C0C0968D939D93D6
:101CC0002F5F243149F74FBF8091E800877F8093D1
:101CD000E8006AE270E0CE0101960E94F00A14C0AA
:101CE000AE014F5F5F4F60911D020E94350ABC013B
:101CF000892B09F440C09091E800977F9093E80009
:101D000089819A810E94530B8091E8008B778093A0
:101D1000E80031C0803879F58091E800877F8093B2
:101D2000E800809114028093F1008091E8008E77A2
:101D30008093E8000E94E90B1EC081111CC09091A5
:101D40001B029230C0F48091E800877F8093E80006
:101D5000909314020E94E90B80911402811106C035
:101D60008091E30087FD02C081E001C084E08093A0
:101D700018020E94FD088091E80083FF0AC080914C
:101D8000E800877F8093E8008091EB008062809379
:101D9000EB00AA960FB6F894DEBF0FBECDBFDF9161
:101DA000CF911F910895CF93809118028823A1F0BD
:101DB000C091E900CF709091EC00892F817090FD67
:101DC00080E8C82B1092E9008091E80083FD0E9412
:101DD000820DCF70C093E900CF91089590938C014C
:101DE00080938B010895E0918B01F0918C013097E5
:101DF00021F00190F081E02D099480E00895EF92A8
:101E0000FF920F931F93CF93DF93E0918B01F0919B
:101E10008C013097B1F18C010280F381E02D09959E
:101E20008091030282FF2DC080FF04C082EA93E00C
:101E30000E947A05E80110E28CE9E82E83E0F82E92
:101E40008091030280FF0BC088811F928F93FF92C5
:101E5000EF920E9413060F900F900F900F90115069
:101E600021961111EDCF8091030280FF0AC08AE90B
:101E700093E0DF91CF911F910F91FF90EF900C9421
:101E80007A05DF91CF911F910F91FF90EF90089508
:101E9000E0918B01F0918C01309721F00480F58165
:101EA000E02D099408952091890130918A018217CB
:101EB000930771F090938A0180938901E0918B01DF
:101EC000F0918C01309721F00680F781E02D099484
:101ED000089520918701309188018217930771F04E
:101EE0009093880180938701E0918B01F0918C01A0
:101EF000309721F00084F185E02D0994089508952C
:101F00000C947F0F0E94881B0C941C06CF92DF92CA
:101F1000EF92FF920F931F93CF93DF9300D000D0E7
:101F200000D0CDB7DEB70E9445068EE8C82E81E00E
:101F3000D82E00E010E0E02E802F0E941E07F60150
:101F400041916F01F42EF826B1F40F5F1F4F00315D
:101F5000110589F78FEF89838A831B820E94911B69
:101F60008160782F9D838C8349815A816B818D811B
:101F70000E94451047C09091030291FF04C08E83D8
:101F80000E9427078E8120E030E04F2D50E0922FF5
:101F9000BA01022E02C0759567950A94E2F760FFB8
:101FA0002BC02983EA8221E030E0690102C0CC0C19
:101FB000DD1C9A95E2F790E08C219D21892B09F494
:101FC00020E02B830E94911B8160782F9D838C835E
:101FD00049815A816B818D810E94451049815A81C6
:101FE0006B817C818D810E940D1BF801E257FE4FB1
:101FF0008081C826C08206C02F5F3F4F2830310540
:1020000031F6A3CF0E940C1B0E94801E10918D01FF
:102010000E94F30E181741F10E94F30E80938D0178
:102020009091030292FF0EC090FF0CC01F928F93FD
:1020300084EB93E09F938F930E9413060F900F9071
:102040000F900F9080918D0126960FB6F894DEBF09
:102050000FBECDBFDF91CF911F910F91FF90EF90F9
:10206000DF90CF900C941E1B26960FB6F894DEBF1F
:102070000FBECDBFDF91CF911F910F91FF90EF90D9
:10208000DF90CF9008950C945507CF93DF93CDB791
:10209000DEB72B970FB6F894DEBF0FBECDBF942FDF
:1020A0004F83252F588769877A878B874A855B8579
:1020B000452B21F02F3F09F59F3FF9F4DE011196E2
:1020C00086E0FD0111928A95E9F785E0FE013796D9
:1020D00001900D928A95E1F749815A816B817C814B
:1020E0008D819E810E9422172B960FB6F894DEBF39
:1020F0000FBECDBFDF91CF9108954F81588569857F
:102100007A858B850E940D1BD9CFCF93882309F444
:10211000A4C0C82F8CEF8C0F813A48F48C2F0E94FA
:10212000CA2181119AC08C2F0E94AD190CC080E287
:102130008C0F883058F4C77081E001C0880FCA95B1
:10214000EAF70E94581ACF910C949C1A8BE58C0FD9
:10215000833078F4C53A29F0C63A31F083E890E04C
:1021600005C081E890E002C082E890E0CF910C9435
:10217000530F88E58C0F853108F06FC0C83A61F1C4
:10218000C93A69F1CA3A71F1CB3A79F1CC3A81F1A5
:10219000CD3A89F1CE3A91F1CF3A99F1C13BA1F113
:1021A000C03BA9F1C23BB1F1C33BB9F1C43BC1F1A2
:1021B000C53BC9F1C63BD1F1C73BD9F1C83BE1F101
:1021C000C93BE9F1CA3BF1F1CB3BF9F1CC3B09F456
:1021D0003FC080E090E03EC082EE90E03BC089EEE0
:1021E00090E038C08AEE90E035C085EB90E032C0D8
:1021F00086EB90E02FC083EB90E02CC084EB90E066
:1022000029C087EB90E026C08CEC90E023C08DECD9
:1022100090E020C083E891E01DC08AE891E01AC0F8
:1022200082E991E017C084E991E014C081E292E074
:1022300011C083E292E00EC084E292E00BC085E21E
:1022400092E008C086E292E005C087E292E002C018
:102250008AE292E0CF910C94690FCF910895882380
:1022600029F19CEF980F913A18F40E94001A0DC0C2
:1022700090E2980F983058F4877091E001C0990F60
:102280008A95EAF7892F0E945E1A0C949C1A9BE5A6
:10229000980F933020F480E090E00C94530F885A0C
:1022A000853120F480E090E00C94690F0895882334
:1022B00021F00E94581A0C949C1A0895882321F04A
:1022C0000E945E1A0C949C1A0895CF92DF92EF92AE
:1022D000FF920F931F93CF93DF9300D000D000D0D5
:1022E000CDB7DEB725E0FC01DE01119601900D921D
:1022F0002A95E1F7FC0140813181F2802581229508
:102300002F7063817481672B09F4D8C23F3F19F4A1
:102310004F3F09F4D3C26C0149833A8389819A8182
:102320002E830E946C19182F092F0E946B190E948E
:102330007B18E02FE295EF70F0E0E05AFF4F2E811E
:102340000C947024802F807F902F9F70092F8823FA
:1023500011F00295007FFF2049F0002309F45FC2CD
:10236000802F0E946B1A0E949C1A59C2812F0E94D2
:102370002F11002309F4A2C2802F0E94711A269601
:102380000FB6F894DEBF0FBECDBFDF91CF911F9186
:102390000F91FF90EF90DF90CF900C949C1A802FBC
:1023A000807F902F9F70092F803211F00295007F5F
:1023B000112319F0113001F129C0FF20A9F0802F5D
:1023C000222349F1213039F526960FB6F894DEBF65
:1023D0000FBECDBFDF91CF911F910F91FF90EF9076
:1023E000DF90CF900C947B1A222319F0213009F44E
:1023F00065C20E94841A2CC0FF20E9F0263008F044
:102400005DC20E94551A802329F022C0FF20F1F0FE
:10241000211115C0802F26960FB6F894DEBF0FBE8F
:10242000CDBFDF91CF911F910F91FF90EF90DF9083
:10243000CF900C945711253008F040C209C0F60126
:10244000858180FFECC18F708583E4CF2111FBC1B2
:10245000802F69C1202F26952695237030E0211505
:10246000310521F021303105C9F028C2FF2021F0CB
:10247000812F902F937002C080E090E026960FB6D7
:10248000F894DEBF0FBECDBFDF91CF911F910F91AA
:10249000FF90EF90DF90CF900C94530FFF2021F02E
:1024A000812F902F937002C080E090E026960FB6A7
:1024B000F894DEBF0FBECDBFDF91CF911F910F917A
:1024C000FF90EF90DF90CF900C94690F812FFF2049
:1024D00019F00E94061D02C00E946E1D26960FB6BE
:1024E000F894DEBF0FBECDBFDF91CF911F910F914A
:1024F000FF90EF90DF90CF900C94F31D802F8370AE
:1025000009F078C0F110DAC1812F82958695877025
:10251000880F880F912F9F70C92ED12CE12CF12CA0
:10252000082E04C0CC0CDD1CEE1CFF1C0A94D2F754
:1025300014FF12C04FE050E060E070E004C0440FB0
:10254000551F661F771F8A95D2F7CB01BA01609598
:1025500070958095909503C060E070E0CB01202FCE
:10256000269526952370422F50E042305105D1F038
:102570004330510559F16C297D298E299F2941301D
:10258000510541F126960FB6F894DEBF0FBECDBFC0
:10259000DF91CF911F910F91FF90EF90DF90CF903F
:1025A0000C9490186C297D298E299F2926960FB6A8
:1025B000F894DEBF0FBECDBFDF91CF911F910F9179
:1025C000FF90EF90DF90CF900C94A2180E9490188B
:1025D000C701B60126960FB6F894DEBF0FBECDBF79
:1025E000DF91CF911F910F91FF90EF90DF90CF90EF
:1025F0000C947E18FF2019F0802F817001C0869501
:10260000882309F45BC1812F829586958770880F96
:10261000880F912F9F70C92ED12CE12CF12C082E00
:1026200004C0CC0CDD1CEE1CFF1C0A94D2F714FF76
:1026300012C04FE050E060E070E004C0440F551F4E
:10264000661F771F8A95D2F7CB01BA016095709506
:102650008095909503C060E070E0CB01202F269517
:1026600026952370422F50E042305105D1F043307F
:10267000510559F16C297D298E299F294130510539
:1026800041F126960FB6F894DEBF0FBECDBFDF91A5
:10269000CF911F910F91FF90EF90DF90CF900C940E
:1026A00047196C297D298E299F2926960FB6F89403
:1026B000DEBF0FBECDBFDF91CF911F910F91FF9075
:1026C000EF90DF90CF900C9459190E944719C701E1
:1026D000B60126960FB6F894DEBF0FBECDBFDF91D0
:1026E000CF911F910F91FF90EF90DF90CF900C94BE
:1026F0003519103F41F118F4103E48F48BC0123FD9
:1027000009F450C0D8F1133F09F460C083C01F70B2
:10271000802F8F71FF2021F00E94CE18812F7BCE59
:102720000E94EF18812F26960FB6F894DEBF0FBED9
:10273000CDBFDF91CF911F910F91FF90EF90DF9070
:10274000CF900C945E11FF20A9F0253008F0B6C0A0
:10275000802F8F7126960FB6F894DEBF0FBECDBFC7
:10276000DF91CF911F910F91FF90EF90DF90CF906D
:102770000C941419263008F0A1C0EACFFF20A1F074
:10278000802F8F7126960FB6F894DEBF0FBECDBF97
:10279000DF91CF911F910F91FF90EF90DF90CF903D
:1027A0000C94CE18FF2061F3802F8F7126960FB600
:1027B000F894DEBF0FBECDBFDF91CF911F910F9177
:1027C000FF90EF90DF90CF900C94EF18FF2091F0E6
:1027D000802F8F7126960FB6F894DEBF0FBECDBF47
:1027E000DF91CF911F910F91FF90EF90DF90CF90ED
:1027F0000C94B91826960FB6F894DEBF0FBECDBF65
:10280000DF91CF911F910F91FF90EF90DF90CF90CC
:102810000C94B418FF20A1F0222309F4B1CF812F2A
:1028200026960FB6F894DEBF0FBECDBFDF91CF91D5
:102830001F910F91FF90EF90DF90CF900C94851037
:10284000222309F4B1CF812F26960FB6F894DEBF6C
:102850000FBECDBFDF91CF911F910F91FF90EF90F1
:10286000DF90CF900C942F11402F4F70612FC60135
:102870000E94801C26960FB6F894DEBF0FBECDBF17
:10288000DF91CF911F910F91FF90EF90DF90CF904C
:102890000C94C617402F4F70612FC60126960FB6B5
:1028A000F894DEBF0FBECDBFDF91CF911F910F9186
:1028B000FF90EF90DF90CF900C94831C26960FB67C
:1028C000F894DEBF0FBECDBFDF91CF911F910F9166
:1028D000FF90EF90DF90CF9008950E94781A0E94A9
:1028E000471A0E949C1A0E94251F0E94F31D80E037
:1028F00090E00E94530F80E090E00C94690F0E94DA
:10290000681A0C946D140E946C19292F22952F704F
:1029100030E02C3031054CF42A3031056CF4225073
:1029200031092230310588F407C02C30310549F0D7
:102930002F30310531F009C0803E48F0803F29F446
:1029400006C093FB882780F9089580E0089581E010
:102950000895CF93DF9300D000D01F92CDB7DEB79C
:102960000F900F900F900F900F90DF91CF910895DF
:10297000CF93DF9300D000D000D0CDB7DEB726963E
:102980000FB6F894DEBF0FBECDBFDF91CF91089593
:102990001F93CF93DF93C0919E0116E080919F011A
:1029A000C81799F0D0E01C9FF0011D9FF00D112475
:1029B000E056FE4F4081518162817381848195810F
:1029C0000E94B8142196C770E9CFDF91CF911F9173
:1029D00008954091D0015091D1016091D201709140
:1029E000D3018091D4019091D5010C94B8148091B9
:1029F000D50182958F7009F054C08091D20188234F
:102A000009F44FC080919E01A0919F016091D00177
:102A10007091D1014091D3015091D401B6E08A1751
:102A200009F43FC090E041155105C1F17F3F11F419
:102A30006F3FA1F1B89FF001B99FF00D1124E0564E
:102A4000FE4F218172132AC02081621327C0228188
:102A5000211124C0238134812417350710F421501B
:102A60003109241B350B2C323140C0F42091D501A3
:102A70002F7020612093D50126E0289FF001299F27
:102A8000F00D1124EB55FE4F80818F7080618083A3
:102A900080ED91E00E9465110C94C8140196877036
:102AA000BECF0895CF92DF92EF92FF920F931F93C4
:102AB000CF93DF93CDB7DEB762970FB6F894DEBF42
:102AC0000FBECDBF8C0185E0F801DE011D9601909F
:102AD0000D928A95E1F7D8014C9111965C9111976E
:102AE00012966C9112971396CD90DC9014973091BA
:102AF000D0017091D1018091D3019091D4010097C0
:102B000009F473C17F3F19F43F3F09F46EC1E090AF
:102B1000D201EE2009F4C5C02091D501C816D9060E
:102B200050F0F601E81BF90BCF01FF24F3948C322F
:102B30009140C8F009C0809590958C0D9D1DFF2493
:102B4000F3948C32914078F0F12C207F09F0C6C0CC
:102B50007C2DD98AC88A89890E94A91480ED91E0C8
:102B60000E946511B1C0822F807F09F045C07513A6
:102B700013C0341311C061110FC02F702061209356
:102B8000D5010E94E91480ED91E00E9465118091C9
:102B9000D501F80185832EC0CD2819F15F3F11F4CE
:102BA0004F3FF9F0F62E61111CC080919E012091DB
:102BB0009F0136E0821709F45BC090E0389FF00176
:102BC000399FF00D1124E056FE4F7181571306C056
:102BD0007081471303C07281711103C00196877021
:102BE000E9CFF62E662309F41DC18091D5018160DD
:102BF0008093D501F12C16C1751309C0341307C099
:102C0000611105C08091D501F8018583C8C04D8749
:102C10005E878D859E856A8B0E9483146A898823CE
:102C2000E1F16623D1F12091D501822F82958F7039
:102C300090E0029774F08091D0019091D101988733
:102C40008F831986DB86CA862C87CE0107960E9461
:102C5000651186E0F801A0EDB1E001900D928A9532
:102C6000E1F70E94F7140E94E914FF24F394DAC0FC
:102C70004D875E878D859E850E946C19292F229530
:102C80002F7030E0223031050CF0BFC09F7009F08A
:102C9000B9C0805E883008F4C5C0C8010E946511C3
:102CA000E4CFC816D90608F453C0F601E81BF90BA7
:102CB000CF018C32914008F453C0F12C7C2DD98A7D
:102CC000C88A89890E94A914E0EDF1E086E0DF015D
:102CD0001D928A95E9F70E94E914A4C0751314C0E7
:102CE000341312C0611110C08091D501F8018583A1
:102CF000C8010E94651186E0E0EDF1E0DF011D9260
:102D00008A95E9F7FE2C8EC04D875E878D859E855E
:102D10006A8B0E9483146A89882309F4BECF6623D4
:102D200009F4BBCF2091D501822F82958F7090E05E
:102D300002970CF48ECF8091D0019091D1019A83AB
:102D400089831B82DD82CC822E83CE0101967FCFC8
:102D5000809590958C0D9D1D8C32914008F0ADCFE3
:102D6000F62E662309F499CF75132EC034132CC0A8
:102D70002091D50120FD1FC0822F82958F70D9F040
:102D8000D80115962C9315978F3049F08F5F982FA7
:102D90009295907F822F8F70892B15968C93C80106
:102DA0000E94651186E0F801A0EDB1E001900D925E
:102DB0008A95E1F790CF86E0F801A0EDB1E00190AF
:102DC0000D928A95E1F72EC04D875E878D859E8591
:102DD0000E94831481113DCF8091D5018160809341
:102DE000D501C8010E9465111DC0662309F455CFA5
:102DF0004D875E878D859E850E948314882309F404
:102E00004CCF27CF811145CF0DC0243031050CF0B8
:102E100044CF9F7009F43DCFD80115969C91907FC7
:102E200009F037CF8F2D62960FB6F894DEBF0FBE34
:102E3000CDBFDF91CF911F910F91FF90EF90DF9069
:102E4000CF9008951F93CF93DF93CDB7DEB72C9724
:102E50000FB6F894DEBF0FBECDBF4F83588769878A
:102E60007A878B879C87CE0107960E94521588230C
:102E700069F08F8198852A853B85232BF1F19F3F4F
:102E800009F063C08F3F09F060C037C086E0FE01E3
:102E90003796DE01119601900D928A95E1F76F81C8
:102EA0007885EA85FB85309741F17F3F11F46F3FCC
:102EB00021F120919F0130E0C90101968770992787
:102EC00040919E0150E08417950709F447C069833B
:102ED0007A83FD83EC8396E0929FD001939FB00D9F
:102EE0001124A056BE4FFE01319601900D929A9585
:102EF000E1F780939F010E94C81416E080919E0123
:102F000090919F018917C1F1189FC001112480562B
:102F10009E4F0E945215882379F1E0919E011E9FD9
:102F2000F0011124E056FE4F40815181628173818E
:102F3000848195810E94B81480919E0190E0019651
:102F40008770992780939E01D9CF4F8158856985D5
:102F50007A858B859C850E94B814CFCF0E947F1400
:102F600010929F0110929E01E0EDF1E086E0DF01FA
:102F70001D928A95E9F7C1CF2C960FB6F894DEBF63
:102F80000FBECDBFDF91CF911F910895DF92EF92D9
:102F9000FF920F931F93CF93DF93FC01892B09F4CA
:102FA0008AC0E12CF12CDD24D394EF012196849189
:102FB000853709F461C058F4843708F04EC0843076
:102FC00008F06AC08130D1F0823071F174C0883766
:102FD00009F45DC050F4863709F455C0873709F00D
:102FE0006AC08E2D0E94651A54C09CE7980F9037D6
:102FF00008F061C08F770E942F1150C08F010E5FC3
:103000001F4FFE01849190E2980F983050F4877022
:10301000FD2D01C0FF0F8A95EAF78F2F0E946B1AD2
:1030200014C00E94851013C08F010E5F1F4FFE0158
:10303000C49180E28C0F883060F4C7708D2D01C080
:10304000880FCA95EAF70E94711A0E949C1AE8013B
:1030500025C08C2F0E942F11FACF9F012E5F3F4F6A
:10306000FE01C491CC2369F08FE99FE00197F1F74D
:1030700000C00000C150F6CF9F012E5F3F4FFE0100
:10308000F490E9010BC00E94551AE82E07C00E9477
:10309000681A0E949C1A02C00E9485108F2D8823F6
:1030A00041F0EFE9FFE03197F1F700C000008150F7
:1030B000F6CFFE017ACFDF91CF911F910F91FF9054
:1030C000EF90DF9008956093DA017093DB018093B5
:1030D000DC019093DD010E941C1B0C946D14609325
:1030E000D6017093D7018093D8019093D9010E94A3
:1030F0001D1B0C946D1408950C9463180F931F936B
:103100000091DA011091DB012091DC013091DD01A9
:10311000602B712B822B932B1F910F910C946318B2
:103120000F931F930091DA011091DB012091DC01D4
:103130003091DD0160237123822393231F910F912E
:103140000C9463180F931F930091DA011091DB0127
:103150002091DC013091DD016027712782279327C0
:103160001F910F910C94631860E070E0CB010C94F8
:103170006F180F931F9341E050E060E070E08A0108
:103180009B0104C0000F111F221F331F8A95D2F725
:10319000C901B8011F910F910C946F180F931F93E1
:1031A00041E050E060E070E004C0440F551F661F2E
:1031B000771F8A95D2F78091D6019091D701A0917F
:1031C000D801B091D9018A019B01082B192B2A2B18
:1031D0003B2BC901B8011F910F910C946F180F93ED
:1031E0001F9341E050E060E070E004C0440F551FC1
:1031F000661F771F8A95D2F7409550956095709518
:103200008091D6019091D701A091D801B091D901B8
:103210008A019B01082319232A233B23C901B801F2
:103220001F910F910C946F180F931F9341E050E082
:1032300060E070E004C0440F551F661F771F8A9539
:10324000D2F78091D6019091D701A091D801B09189
:10325000D9018A019B01082719272A273B27C90181
:10326000B8011F910F910C946F180F931F93009149
:10327000D6011091D7012091D8013091D901602B4E
:10328000712B822B932B1F910F910C946F180F931E
:103290001F930091D6011091D7012091D801309150
:1032A000D90160237123822393231F910F910C94E2
:1032B0006F180F931F930091D6011091D7012091A1
:1032C000D8013091D90160277127822793271F9158
:1032D0000F910C946F180895CF92DF92EF92FF92A6
:1032E0000F931F93CF93DF938C01C090DA01D0909E
:1032F000DB01E090DC01F090DD014091D6015091BE
:10330000D7016091D8017091D901C42AD52AE62A43
:10331000F72ACFE1D0E0D701C6010C2E04C0B69544
:10332000A795979587950A94D2F780FF07C0B801B3
:103330008C2F0E94551C8130910531F4219758F74C
:10334000B80180E00E94551CDF91CF911F910F9131
:10335000FF90EF90DF90CF90089590910A0199230C
:1033600021F090910B01911109C020910C01309135
:103370000D01F90132969FEF40E030C0982F9695ED
:10338000969596959F31A0F4E0910C01F0910D0176
:10339000E90FF11D877021E030E0A90102C0440F60
:1033A000551F8A95E2F7CA019181892B818308957F
:1033B0009091030290FF23C01F928F938DED93E0B5
:1033C0009F938F930E9413060F900F900F900F9072
:1033D00008959F3F39F04F5F4E3141F0519158139E
:1033E000F8CF0DC05111F7CF942FF5CF9F3F39F093
:1033F000F901E90FF11D97FDFA958283089508956B
:1034000090910A01992321F090910B01911109C02B
:1034100020910C0130910D01F9013296205E3F4F51
:1034200030C0982F9695969596959F31A8F4E09187
:103430000C01F0910D01E90FF11D877021E030E0E2
:10344000A90102C0440F551F8A95E2F7CA01809571
:1034500091818923818308959091030290FF16C082
:103460001F928F938FEB93E09F938F930E9413068D
:103470000F900F900F900F9008953196E217F30779
:1034800029F090819813F9CF1082F7CF089581E049
:1034900090E0E0910C01F0910D01E80FF91F10820E
:1034A000019680329105A9F708958091020208954E
:1034B00090910202892B8093020208958095909149
:1034C00002028923809302020895809302020895E4
:1034D00010920202089590910102892B80930102BB
:1034E00008958095909101028923809301020895A7
:1034F0001092010208958093E0010E94911B909325
:10350000DF018093DE0108951092E0011092DF0147
:103510001092DE01089580910C0190910D01FC0143
:1035200031969C01205E3F4F80E0919191118F5F19
:10353000E217F307D1F70895E0910C01F0910D0126
:10354000809102028083E0910C01F0910D01908145
:1035500080910102892B80838091E0018823D9F139
:103560000E94911B2091DE013091DF0182179307A9
:1035700048F00E94911B2091DE013091DF01821BF7
:10358000930B0AC00E94911B2091DE013091DF0154
:1035900020953095820F931F8C32914070F080916E
:1035A000030280FF08C08BEF93E09F938F930E94EC
:1035B00013060F900F900E94841AE0910C01F09175
:1035C0000D0190818091E001892B80830E948B1AEC
:1035D00081110E94841A80910C0190910D010C942C
:1035E000FF0E909339018093380108958295982FAA
:1035F0009C7C392F36953695282F237344E0249FE1
:10360000C0011124932F982B292F2A7A2695892FD0
:103610008575880F822B08950895CF93DF9300D08E
:1036200000D01F92CDB7DEB70F900F900F900F9084
:103630000F90DF91CF910895089508950C94431051
:1036400080911802843021F11092040220E488E174
:1036500090E00FB6F894A895809360000FBE209379
:10366000600083B7817F846083BF83B7816083BF3D
:103670007894889583B78E7F83BF0FB6F894A8950A
:1036800080916000886180936000109260000FBE9E
:103690000895CF930E9453070E9445060E94540745
:1036A000C0E08C2F0E941E07811104C0CF5FC03183
:1036B000C1F701C081E0CF9108950C947F141F924F
:1036C0000F920FB60F9211248F939F93AF93BF93D6
:1036D00080910402811113C080910502909106022D
:1036E000A0910702B09108024196A11DB11D8093DF
:1036F000050290930602A0930702B0930802BF91BF
:10370000AF919F918F910F900FBE0F901F901895C2
:1037100082E084BD93E095BD9AEF97BD80936E00E3
:1037200008952FB7F8948091050290910602A09118
:103730000702B09108022FBF08952FB7F894609147
:1037400005027091060280910702909108022FBF36
:103750000895CF92DF92EF92FF920F931F932FB7AE
:10376000F894409105025091060260910702709111
:1037700008022FBF6A017B01EE24FF248C0120E0A8
:1037800030E0C016D106E206F30610F441505109AC
:103790009A01281B390BC9011F910F91FF90EF90DF
:1037A000DF90CF900895CF92DF92EF92FF920F9328
:1037B0001F932FB7F894C0900502D0900602E090B6
:1037C0000702F09008022FBF97018601061B170B16
:1037D000280B390BC616D706E806F90618F0C901FA
:1037E000B80106C0C901B801615071098109910988
:1037F0001F910F91FF90EF90DF90CF9008951F924F
:103800000F920FB60F9211248F939F93AF93BF9394
:103810008091050290910602A0910702B0910802E2
:103820000196A11DB11D8093050290930602A093FD
:103830000702B0930802BF91AF919F918F910F90B3
:103840000FBE0F901F9018950E943A0CF8942FEF1E
:1038500087EA91E6215080409040E1F700C00000E7
:1038600087E090EBDC018093210290932202A093E9
:103870002302B09324029CE088E10FB6F894A89547
:10388000809360000FBE90936000FFCF28E0929F6E
:10389000F0011124E80FF11DE052FF4F8491982FA1
:1038A00090778F7092959F700895CF93C82FCB011A
:1038B0000E94461C292F30E0E82FF0E0A90164E0C7
:1038C000440F551F6A95E1F74E2B5F2B4038510589
:1038D00019F480E090E012C088E0C89F200D311DEF
:1038E000112484E0220F331F8A95E1F7E20FF31FC2
:1038F000EE0FFF1FE050F84985919491CF91089504
:1039000080E090E00895089580910B0280FF0BC045
:103910006091110185E0689FB0011124759567954C
:10392000759567952BC081FF09C06091110185E0F5
:10393000689FB00111247595679520C082FF07C06C
:103940006091110185E0689FB001112417C090912A
:103950000C029923D1F060911001961788F72091FD
:10396000110185E0289F90011124929FA001939F4F
:10397000500D112470E0CA010E945C24603871056A
:1039800040F46115710539F002C065E070E0862FE2
:1039900008958FE7089581E0089580910B0280FFDC
:1039A00008C060910F0170E07595679575956795F2
:1039B00021C081FF06C060910F0170E07595679589
:1039C00019C082FF04C060910F0170E010C0909197
:1039D0000C029923C1F060910E019617A0F7809117
:1039E0000F01899FC001112470E00E945C2460389F
:1039F000710528F46115710521F0862F08958FE770
:103A0000089581E0089561E070E0F4CF803F21F4F3
:103A10000E94841C819504C0813F29F40E94841C6B
:103A200080930F020895823F21F40E94841C8195A7
:103A300004C0833F29F40E94841C80930E020895E1
:103A4000893F19F40E94CD1C05C08A3F31F40E94C1
:103A5000CD1C81958093100208958B3F21F40E9424
:103A6000CD1C819504C08C3F29F40E94CD1C80930D
:103A700011020895843F21F480910D02816017C0E6
:103A8000853F21F480910D02826011C0863F21F4B0
:103A900080910D0284600BC0873F21F480910D025C
:103AA000886005C0883F31F480910D028061809369
:103AB0000D0208958D3F21F480910B0281600BC0AF
:103AC0008E3F21F480910B02826005C08F3F29F464
:103AD00080910B02846080930B020895803F39F43B
:103AE00080910F0287FF6CC010920F0269C0813F66
:103AF00029F480910F021816BCF362C090910E0257
:103B0000823F29F497FF5CC010920E0259C0833F98
:103B100019F41916CCF354C0893F41F48091100276
:103B200018160CF04DC0109210024AC08A3F29F4BA
:103B30008091100287FF44C0F6CF8B3F39F480910B
:103B4000110287FF3DC0109211023AC08C3F29F448
:103B5000809111021816BCF333C0843F21F4809188
:103B60000D028E7F17C0853F21F480910D028D7F5D
:103B700011C0863F21F480910D028B7F0BC0873FDF
:103B800021F480910D02877F05C0883F31F4809138
:103B90000D028F7E80930D0213C08D3F21F4809122
:103BA0000B028E7F0BC08E3F21F480910B028D7F24
:103BB00005C08F3F29F480910B028B7F80930B020D
:103BC00080910E0281110EC080910F0281110AC0F6
:103BD00080911002811106C080911102811102C0F2
:103BE00010920C0208958091030283FF7EC084E34B
:103BF00094E00E947A0580910D021F928F938FE2CC
:103C000094E09F938F930E9413068DE294E00E94AC
:103C10007A0580910E02282F082E000C330B3F935B
:103C20008F938AE294E09F938F930E94130688E219
:103C300094E00E947A0580910F02282F082E000C34
:103C4000330B3F938F9385E294E09F938F930E9471
:103C5000130683E294E00E947A0580911002282FD7
:103C6000082E000C330B3F938F9380E294E09F93D8
:103C70008F930E9413068EE194E00E947A05809152
:103C80001102282F082E000C330B3F938F938BE1EA
:103C900094E09F938F930E94130688E194E00E9422
:103CA0007A0580910C021F928F9385E194E09F9397
:103CB0008F930E94130683E194E00E947A0580911D
:103CC0000B021F928F9380E194E09F938F930E9449
:103CD00013068DE094E00E947A058DB79EB74C964E
:103CE0000FB6F8949EBF0FBE8DBF8DE092E00E948C
:103CF000480F0E94911B90930A0280930902089535
:103D00001F93CF93DF938091090290910A020E9442
:103D1000A91BAC0190910C02992321F02091120172
:103D200030E006C0209113018AE0289F9001112401
:103D30004217530708F485C080910E02C0910F020C
:103D4000D091100210911102811107C0C11175C0EC
:103D5000D11173C0111171C074C09F3F19F09F5FE2
:103D600090930C02181624F40E94841C80930E0277
:103D700080910E0287FF05C00E94841C819580936C
:103D80000E021C1624F40E94841C80930F02809162
:103D90000F0287FF05C00E94841C819580930F024B
:103DA00060910E02662331F1C0910F02CC2311F114
:103DB000062E000C770B880B990B0E94572323E3E8
:103DC00033E343E35FE30E94BB230E941F2360931E
:103DD0000E026C2FCC0F770B880B990B0E94572388
:103DE00023E333E343E35FE30E94BB230E941F23EB
:103DF00060930F021D1624F40E94CD1C80931002C4
:103E00008091100287FF05C00E94CD1C8195809390
:103E10001002111624F40E94CD1C8093110280918F
:103E2000110287FF05C00E94CD1C8195809311026D
:103E3000DF91CF911F910C94F31D9F3F09F08FCF1D
:103E400097CFDF91CF911F910895EDE0F2E085E0EB
:103E5000DF011D928A95E9F710920C0210920B0275
:103E6000089587E596E00E947A051F9281E08F937E
:103E70001F9285E08F9389E096E09F938F930E9435
:103E800013060F900F900F900F900F900F900895C2
:103E90008330E9F128F4813061F0823009F108952E
:103EA000853009F462C008F449C0863009F474C052
:103EB000089580911301262F30E0280F311D2F3FE8
:103EC000310524F4680F6093130103C08FEF8093D2
:103ED0001301809113011F928F9382E495E072C0C9
:103EE00080911201262F30E0280F311D2F3F310520
:103EF00024F4680F6093120103C08FEF80931201C6
:103F0000809112011F928F9380E395E05BC08091B6
:103F10001101262F30E0280F311D2F3F310524F4E9
:103F2000680F6093110103C08FEF8093110180919E
:103F300011011F928F938DE195E044C08091100193
:103F4000262F30E0280F311D2F3F310524F4680F54
:103F50006093100103C08FEF8093100180911001D6
:103F60001F928F9388E095E02DC080910F01262F3E
:103F700030E0280F311D2F3F310524F4680F609386
:103F80000F0103C08FEF80930F0180910F011F92EB
:103F90008F938FEE94E016C080910E01262F30E0B3
:103FA000280F311D2F3F310524F4680F60930E0157
:103FB00003C08FEF80930E0180910E011F928F93AB
:103FC00084ED94E09F938F930E9413060F900F90BF
:103FD0000F900F900895833081F128F4813059F0CB
:103FE0008230D1F00895853009F449C0B8F18630A7
:103FF00009F456C0089580911301681720F4861BB8
:104000008093130102C010921301809113011F923B
:104010008F9385EC94E054C080911201681720F4CE
:10402000861B8093120102C010921201809112012E
:104030001F928F9383EB94E043C080911101681726
:1040400020F4861B8093110102C01092110180910F
:1040500011011F928F9380EA94E032C08091100189
:10406000681720F4861B8093100102C01092100183
:10407000809110011F928F938BE894E021C0809172
:104080000F01681720F4861B80930F0102C0109265
:104090000F0180910F011F928F9382E794E010C06F
:1040A00080910E01681720F4861B80930E0102C0D8
:1040B00010920E0180910E011F928F9387E594E07C
:1040C0009F938F930E9413060F900F900F900F9065
:1040D0000895CF93C82F1F928F938CE597E09F93FD
:1040E0008F930E94130681E090E0A0E0B0E0BC0155
:1040F000CD0104C0660F771F881F991FCA95D2F79C
:104100000E947C180F900F900F900F90CF910C94FD
:104110007F14CF938732A8F58E3108F02BC1803100
:1041200009F49FC0F8F4873009F464C0A8F486301D
:1041300009F024C180910302817F8E7F8093030266
:1041400081E697E00E947A0585E49AE00E947A056C
:1041500081E0809313024CC08B30F1F18E3009F472
:104160006CC00CC1863109F4B0C020F4813109F46F
:10417000EDC004C1893109F491C08B3109F449C003
:10418000FDC0883349F150F4893209F4F1C0853318
:1041900009F4EEC0873209F0F1C0EAC0833409F4B3
:1041A000E7C028F48A3308F4E9C08953E4C08834AE
:1041B00009F0E4C00E947F1484E39AE00E947A052B
:1041C0002FEF83ED90E3215080409040E1F700C055
:1041D00000000E94241C0CC088E897E05CC08BE1C2
:1041E0009AE00E947A058091030281608093030225
:1041F000C1E0C9C080910302C82FC17080FFEFCF1A
:1042000087E29AE00E947A0580910302817F8E7F87
:104210003DC09091030291FBCC27C0F981E0C827F3
:10422000892FC0FB81F980930302CC2319F08EE023
:104230009AE027C080E09AE02EC09091030292FBA2
:10424000CC27C0F981E0C827892FC0FB82F9809371
:104250000302CC2319F081EF99E013C081EE99E0BD
:104260001AC09091030293FBCC27C0F981E0C827C4
:10427000892FC0FB83F980930302CC2351F085ED95
:1042800099E00E947A058091030281608093030285
:104290007AC088EC99E00E947A05AACF89EB99E070
:1042A0000E947A058CE899E00E947A0585E599E0FC
:1042B0000E947A058EE299E00E947A0584EE98E0E9
:1042C0000E947A0586EB98E0E6CF88EA98E00E94A3
:1042D0007A050E94F30E1F928F938EE898E09F93C9
:1042E0008F930E94130680910A011F928F9387E794
:1042F00098E09F938F930E941306809186011F92EE
:104300008F9384E698E09F938F930E941306809189
:104310000B011F928F9381E598E09F938F930E94EA
:1043200013060E949D1B9F938F937F936F938AE345
:1043300098E09F938F930E9413068DB79EB7469681
:104340000FB6F8949EBF0FBE8DBF52CF0E947F1450
:10435000C0910B0181E0C827C0930B01CC2329F049
:1043600080E398E00E947A050EC085E298E093CF42
:1043700080E001C08D510E9469203ACF83E298E02D
:104380000E947A05C0E08C2FCF91089580E00895B7
:1043900080E00895CF93C82F80911302813071F08F
:1043A00020F0823009F44BC042C1E0910C01F09141
:1043B0000D018081823209F03CC107C0E0910C01FF
:1043C000F0910D018081823261F48C2F0E94C62110
:1043D000811104C08C2F0E9489202FC081E090E0C1
:1043E0002CC08C2F0E94C821811126C0C431E1F05D
:1043F00070F4CB3081F0C031D1F40E94311F84E5DC
:1044000097E00E947A0582E08093130215C0C932BA
:1044100059F0C83361F481E697E00E947A0588E597
:1044200097E00E947A0508C01092130204C182E549
:1044300097E00E947A05FFC081E08170FEC0C4321F
:1044400028F5CE3108F0C1C0CB30A1F1D0F4C7308F
:1044500009F0D3C08EE18093130182E380931201AF
:104460008AE08093110184E18093100188E08093B9
:104470000F0188E280930E0188EF95E00E947A0593
:10448000BFC0C33149F1C431C1F0B7C0CB3409F466
:10449000A9C028F4C93289F0C83361F0AEC0C13573
:1044A00009F49EC0C23509F499C0CE3409F0A5C004
:1044B0006AE09EC00E94311FA3C08091120288232F
:1044C00019F0109212029CC085E096E00E947A05D5
:1044D00081E080931302B1C08FED95E00E947A05D0
:1044E0008DEC95E00E947A05809113011F928F93C5
:1044F0008AEC95E09F938F930E94130688EC95E0D9
:104500000E947A0586EB95E00E947A05809112015F
:104510001F928F9383EB95E09F938F930E941306D6
:1045200081EB95E00E947A0582EA95E00E947A0587
:10453000809111011F928F938FE995E09F938F9344
:104540000E9413068DE995E00E947A058CE895E0BB
:104550000E947A05809110011F928F9389E895E05F
:104560009F938F930E94130687E895E00E947A0537
:1045700082E795E00E947A0580910F011F928F9348
:104580008FE695E09F938F930E9413068DE695E04A
:104590000E947A0586E595E00E947A0580910E01D9
:1045A0001F928F9383E595E09F938F930E9413064C
:1045B00081E595E00E947A058DB79EB748960FB6C3
:1045C000F8949EBF0FBE8DBF1BC0CE51EC2FF0E004
:1045D000E35DFE4F80818093120212C061E003C050
:1045E00061E006C06AE0809112020E94481F08C084
:1045F000809112020E94EB1F03C086EF95E013C06A
:1046000080911202882369F01F928F9380EF95E0CA
:104610009F938F930E9413060F900F900F900F900F
:1046200004C08DEE95E00E947A0581E006C01092EC
:10463000130280E002C080E000CFCF9108950E9475
:1046400026236894B1110C94B52308950E949A23EF
:1046500088F09F5798F0B92F9927B751B0F0E1F043
:10466000660F771F881F991F1AF0BA95C9F714C0F3
:10467000B13091F00E94B423B1E008950C94B423BA
:10468000672F782F8827B85F39F0B93FCCF386952C
:1046900077956795B395D9F73EF490958095709589
:1046A00061957F4F8F4F9F4F0895E89409C097FB06
:1046B0003EF490958095709561957F4F8F4F9F4FF9
:1046C0009923A9F0F92F96E9BB279395F69587953D
:1046D00077956795B795F111F8CFFAF4BB0F11F400
:1046E00060FF1BC06F5F7F4F8F4F9F4F16C08823A7
:1046F00011F096E911C0772321F09EE8872F762FDD
:1047000005C0662371F096E8862F70E060E02AF01D
:104710009A95660F771F881FDAF7880F9695879509
:1047200097F9089557FD9058440F551F59F05F3F72
:1047300071F04795880F97FB991F61F09F3F79F0C3
:1047400087950895121613061406551FF2CF469545
:10475000F1DF08C0161617061806991FF1CF8695C7
:104760007105610508940895E894BB2766277727AB
:10477000CB0197F908950E94CE230C943F240E9408
:10478000312438F00E94382420F0952311F00C9445
:1047900028240C942E2411240C94B5230E949223D7
:1047A00070F3959FC1F3950F50E0551F629FF00184
:1047B000729FBB27F00DB11D639FAA27F00DB11D9D
:1047C000AA1F649F6627B00DA11D661F829F222726
:1047D000B00DA11D621F739FB00DA11D621F839FAD
:1047E000A00D611D221F749F3327A00D611D231F83
:1047F000849F600D211D822F762F6A2F11249F57D1
:1048000050409AF0F1F088234AF0EE0FFF1FBB1FD3
:10481000661F771F881F91505040A9F79E3F510592
:1048200080F00C9428240C94B5235F3FE4F3983E69
:10483000D4F3869577956795B795F795E7959F5F3C
:10484000C1F7FE2B880F911D9695879597F90895CE
:1048500097F99F6780E870E060E008959FEF80EC33
:10486000089500240A9416161706180609060895D6
:1048700000240A9412161306140605060895092E3C
:104880000394000C11F4882352F0BB0F40F4BF2BAB
:1048900011F460FF04C06F5F7F4F8F4F9F4F0895EB
:1048A000991B79E004C0991F961708F0961B881F82
:1048B0007A95C9F78095089597FB072E16F4009412
:1048C00007D077FD09D00E94762407FC05D03EF47E
:1048D000909581959F4F0895709561957F4F0895AC
:1048E000EE0FFF1F0590F491E02D0994AA1BBB1B4E
:1048F00051E107C0AA1FBB1FA617B70710F0A61BE0
:10490000B70B881F991F5A95A9F780959095BC0100
:08491000CD010895F894FFCFDA
:104918005C074D082A08F607C2070101E1012808CB
:10492800140A321E404D3622395A030D03D702B5F8
:10493800027C02EF01080221023A025A0201020334
:08494800040506070809000040
:1068000088000000000000000400050006000700EA
:10681000080009000A000B000C000D000E000F001C
:1068200010001100120013001400150016001700CC
:10683000180019001A001B001C001D001E001F007C
:10684000200021002200230024002500260027002C
:10685000280035002A002B002C002D002E002F00D0
:1068600030000000320033003400290036003700C9
:106870003800E00000000000000000000000000000
:106880000000000000000000000000000000000008
:1068900000000000000000000000000000004F00A9
:1068A00050005100520000000000000000000000F5
:1068B00000000000000000000000000000000000D8
:1068C00000000000000000000000000000000000C8
:1068D00000000000000000000000000000000000B8
:1068E0000000000000000000890087008A008B0083
:1068F000F1A1E100E200E300F1A1E500E600000003
:106900000100010001000100EA4401000100E2442D
:106910000100010001005500460054004A004B00F0
:10692000560057004700480001000100E9440100FB
:106930000100010001000100010001003A003B00DC
:106940003C003D003E003F0040004100420043004B
:10695000580001004C00390001004400450052007D
:1069600001000100010050004F0081404D004E0029
:1069700051000100010001000100010001000100BF
:1069800001000100010001000100010001000100FF
:1069900001000100010001000100010001004D00A3
:1069A0004A004E004B0001000100010001000100FF
:1069B00001000100010001000100010001000100CF
:1069C00001000100010001000100010001000100BF
:1069D00001000100010001000100010001000100AF
:1069E0000100010001000100490001000100010057
:1069F000010001000100010001000100010001008F
:00000001FF
